:10000000000000308A002B28A501A400FF30A407BF
:10001000031CA507031C26280330A300DF30122091
:100020000628A301E83EA200A309FC30031C1B28FC
:10003000A20703181828A2070000A30F18282218E7
:100040002128A21C252800002528080083138312DC
:100050000313000008000130A500F4308A010520D8
:10006000831685013F3086008701880183128A1537
:100070000A12B4238A110A12AA248A110A12061C2F
:1000800044288A150A12D1298A110A1206194B2806
:100090008A110A12BB2F8A110A12861852288A1155
:1000A0000A12222DA101A0018A110A12BA2A0030D7
:1000B00021078A006230200703188A0AA00A031960
:1000C000A10A8200013400340034003400340034CA
:1000D000003400340034003402340034003400347E
:1000E000003400340034003400340034043400346C
:1000F0000034003400340034003400340034003460
:100100000834003400340034003400340034003447
:10011000003400341034003400340034003400342F
:10012000003400340034003420340034003400340F
:10013000003400340034003400340034003401341E
:10014000003400340034003400340034003400340F
:1001500000340234003400340034003400340034FD
:1001600000340034003404340034003400340034EB
:1001700000340034003400340034083400340034D7
:1001800000340034003400340034003400341034BF
:1001900000340034003400340034003400340034BF
:1001A000003420340034003400340034003400348F
:1001B000003400340034003401340034003400349E
:1001C000003400340034003400340034023400348D
:1001D000003400340034003400340034003400347F
:1001E000043400340034003400340034003400346B
:1001F0000034003408340034003400340034003457
:10020000003400340034003410340034003400343E
:10021000003400340034003400340034203400341E
:10022000003400340034003400340034003400342E
:10023000003401340034003400340034003400341D
:10024000003400340034023400340034003400340C
:1002500000340034003400340034043400340034FA
:1002600000340034003400340034003400340834E6
:1002700000340034003400340034003400340034DE
:1002800000341034003400340034003400340034BE
:10029000003400340034203400340034003400349E
:1002A00000340034003400340034003401340034AD
:1002B000003400340034003400340034003400349E
:1002C000023400340034003400340034003400348C
:1002D000003400340434003400340034003400347A
:1002E0000034003400340034083400340034003466
:1002F000003400340034003400340034103400344E
:10030000003400340034003400340034003400344D
:10031000203400340034003400340034003400341D
:10032000003400340034013400340034003400342C
:10033000003400340034003400340234003400341B
:100340000034003400340034003400340034043409
:1003500000340034003400340034003400340034FD
:1003600000340834003400340034003400340034E5
:1003700000340034003410340034003400340034CD
:1003800000340034003400340034203400340034AD
:1003900000340034003400340034003400340034BD
:1003A00001340034003400340034003400340034AC
:1003B000003400340234003400340034003400349B
:1003C0000034003400340034043400340034003489
:1003D0000034003400340034003400340834003475
:1003E000003400340034003400340034003400346D
:1003F000103400340034003400340034003400344D
:10040000003400342034003400340034003400342C
:10041000003400340034003400340134003400343B
:10042000003400340034003400340034003402342A
:10043000003400340034003400340034003400341C
:100440000034043400340034003400340034003408
:1004500000340034003408340034003400340034F4
:1004600000340034003400340034103400340034DC
:1004700000340034003400340034003400342034BC
:1004800000340034003400340034003400340034CC
:1004900000340034013400340034003400340034BB
:1004A00000340034003400340234003400340034AA
:1004B0000034003400340034003400340434003498
:1004C000003400340034003400340034003400348C
:1004D0000834003400340034003400340034003474
:1004E000003400341034003400340034003400345C
:1004F000003400340034003420340034003400343C
:10050000003400340034003400340034003401344A
:10051000003400340034003400340034003400343B
:100520000034023400340034003400340034003429
:100530000034003400340434003400340034003417
:100540000034003400340034003408340034003403
:1005500000340034003400340034003400341034EB
:1005600000340034003400340034003400340034EB
:1005700000342034BF013F088A110A12031DC12A2A
:10058000B00A8A015720A6008A015720A7008A01D5
:100590005720A8008A015720A9008A015720AA00E5
:1005A0008A015720AB008A015720AC008A015720EE
:1005B000AD008A015720AE008A015720AF00BE0A65
:1005C0008A110A128618E72A8A110A12222D320885
:1005D000870005308A0104202608870005308A013B
:1005E0000420403087003308870005308A0104204A
:1005F0002708870005308A0104204030870034082E
:10060000870005308A010420280887001130A300E4
:1006100034308A01122040308700350887000530C9
:100620008A0104202908870005308A01042040300F
:1006300087003608870005308A0104202A088700D1
:1006400005308A01042040308700370887000530D4
:100650008A0104202B08870005308A0104204030DD
:1006600087003808870005308A0104202C0887009D
:1006700005308A01042040308700390887000530A2
:100680008A0104202D08870005308A0104204030AB
:1006900087003A08870005308A0104202E08870069
:1006A00005308A010420403087003B088700053070
:1006B0008A0104202F08870005308A010420803039
:1006C000870087018A110A12AA243D3030028A115C
:1006D0000A12031D6E2B8A110A12962B3C303E0221
:1006E0008A110A12031D762BA101A0013C303E02A3
:1006F0008A110A12031D7D2BBE01BF0A32303F0250
:100700008A110A12031D862B8A01BA2A8A110A123B
:1007100006198D2B8A110A12BB2F8A110A12061C88
:10072000942B8A150A12D1298A01E72AB001BF0148
:10073000BE01A101A0010310B20D403032028A11A6
:100740000A12031DA62B8A110A120B2C0310B30DDB
:10075000403033028A110A12031DB12B8A110A128A
:100760000B2C0310B40D403034028A110A12031D01
:10077000BC2B8A110A120B2C0310B50D4030350228
:100780008A110A12031DC72B8A110A120B2C03109F
:10079000B60D403036028A110A12031DD22B8A117F
:1007A0000A120B2C0310B70D403037028A110A12BF
:1007B000031DDD2B8A110A120B2C0310B80D4030DB
:1007C00038028A110A12031DE82B8A110A120B2C17
:1007D0000310B90D403039028A110A12031DF32BA0
:1007E0008A110A120B2C0310BA0D40303A028A11FA
:1007F0000A12031DFE2B8A110A120B2C0310BB0DCB
:1008000040303B028A110A12031D092C8A110A1278
:100810000B2C8A01BA2A403032028A110A12031DB7
:10082000132C0130B300403032028A110A12031D2A
:100830001A2CB201403033028A110A12031D222CF5
:100840000130B400403033028A110A12031D292CF2
:10085000B301403034028A110A12031D312C0130D9
:10086000B500403034028A110A12031D382CB4013D
:10087000403035028A110A12031D402C0130B600A7
:10088000403035028A110A12031D472CB501403051
:1008900036028A110A12031D4F2C0130B700403076
:1008A00036028A110A12031D562CB6014030370257
:1008B0008A110A12031D5E2C0130B8004030370245
:1008C0008A110A12031D652CB701403038028A11C3
:1008D0000A12031D6D2C0130B900403038028A1114
:1008E0000A12031D742CB801403039028A110A1211
:1008F000031D7C2C0130BA00403039028A110A12E3
:10090000031D832CB90140303A028A110A12031DDB
:100910008B2C0130BB0040303A028A110A12031DB1
:10092000922CBA0140303B028A110A12031D9A2C04
:100930000130B200013032028A110A12031DA12CCB
:10094000BD0A40303B028A110A12031DA82CBB01CC
:100950008A01BA2A0D303D028A110A12031DB22CF7
:100960000130BD0001303D028A110A12031DBA2C6C
:100970000130880002303D028A110A12031DC22C88
:100980000230880003303D028A110A12031DCA2C6E
:100990000430880004303D028A110A12031DD22C53
:1009A0000830880005303D028A110A12031DDA2C36
:1009B0001030880006303D028A110A12031DE22C15
:1009C0002030880007303D028A110A12031DEA2CEC
:1009D0004030880008303D028A110A12031DF22CB3
:1009E0008030880009303D028A110A12031CF92C5C
:1009F000880109303D028A110A12031D012D313090
:100A000085000A303D028A110A12031D092D323079
:100A100085000B303D028A110A12031D112D34305E
:100A200085000C303D028A110A12031D192D383041
:100A3000850009303D028A110A120318212D303039
:100A400085000800320887000A308A0104204030FF
:100A50008700330887000A308A010420403087006D
:100A60003408870009308A010420403087003508A7
:100A700087000A308A01042040308700360887004A
:100A80000A308A01042040308700370887000A3086
:100A90008A01042040308700380887000A308A0124
:100AA000042040308700390887000A308A0104207A
:100AB000403087003A0887000A308A01042040301D
:100AC00087003B0887002230A300FE308A011220F5
:100AD0008030870087013D3030028A110A12031DE1
:100AE000742D8A110A12B82DBF0AB10A32303F02A2
:100AF0008A110A12031D7D2DB00A323031028A118B
:100B00000A120318862D8A110A12CC2633303102BC
:100B10008A110A12031C8F2D8A110A1244273230BF
:100B20003F028A110A12031D962DBF016530310262
:100B30008A110A12031C9D2DB1018A110A1206198D
:100B4000A42D8A110A12BB2F8A110A12061CAB2D82
:100B50008A150A12D1298A110A12861CB02DB001F9
:100B60008A110A12861CB62D8A01BA2A8A01222D00
:100B7000B001BF01BE01A101A0010310B20D4030C0
:100B800032028A110A12031DC82D8A110A122D2E53
:100B90000310B30D403033028A110A12031DD32D06
:100BA0008A110A122D2E0310B40D403034028A111E
:100BB0000A12031DDE2D8A110A122D2E0310B50D07
:100BC000403035028A110A12031DE92D8A110A12DA
:100BD0002D2E0310B60D403036028A110A12031D65
:100BE000F42D8A110A122D2E0310B70D4030370252
:100BF0008A110A12031DFF2D8A110A122D2E0310CD
:100C0000B80D403038028A110A12031D0A2E8A11CB
:100C10000A122D2E0310B90D403039028A110A1222
:100C2000031D152E8A110A122D2E0310BA0D403005
:100C30003A028A110A12031D202E8A110A122D2E41
:100C40000310BB0D40303B028A110A12031D2B2EEC
:100C50008A110A122D2E8A01222D403032028A1169
:100C60000A12031D352E0130B300403032028A11C2
:100C70000A12031D3C2EB201403033028A110A12BF
:100C8000031D442E0130B400403033028A110A1291
:100C9000031D4B2EB301403034028A110A12031D8A
:100CA000532E0130B500403034028A110A12031D60
:100CB0005A2EB401403035028A110A12031D622EE9
:100CC0000130B600403035028A110A12031D692E28
:100CD000B501403036028A110A12031D712E01300F
:100CE000B700403036028A110A12031D782EB60171
:100CF000403037028A110A12031D802E0130B800DD
:100D0000403037028A110A12031D872EB701403086
:100D100038028A110A12031D8F2E0130B9004030AB
:100D200038028A110A12031D962EB801403039028A
:100D30008A110A12031D9E2E0130BA00403039027A
:100D40008A110A12031DA52EB90140303A028A11F8
:100D50000A12031DAD2E0130BB0040303A028A1149
:100D60000A12031DB42EBA0140303B028A110A1246
:100D7000031DBC2E0130B200013032028A110A126A
:100D8000031DC32EBD0A40303B028A110A12031D07
:100D9000CA2EBB018A01222D0D303D028A110A1292
:100DA000031DD42E0130BD0001303D028A110A120C
:100DB000031DDC2E0130880002303D028A110A1228
:100DC000031DE42E0230880003303D028A110A120E
:100DD000031DEC2E0430880004303D028A110A12F3
:100DE000031DF42E0830880005303D028A110A12D6
:100DF000031DFC2E1030880006303D028A110A12B5
:100E0000031D042F2030880007303D028A110A128A
:100E1000031D0C2F4030880008303D028A110A1251
:100E2000031D142F8030880009303D028A110A12F8
:100E3000031C1B2F880109303D028A110A12031D71
:100E4000232F213085000A303D028A110A12031D2A
:100E50002B2F223085000B303D028A110A12031D10
:100E6000332F243085000C303D028A110A12031DF5
:100E70003B2F2830850009303D028A110A120318E1
:100E8000432F2030850008000D303D028A110A12E0
:100E9000031D4C2F0130BD0001303D028A110A12A2
:100EA000031D542F0130880002303D028A110A12BE
:100EB000031D5C2F0230880003303D028A110A12A4
:100EC000031D642F0430880004303D028A110A1289
:100ED000031D6C2F0830880005303D028A110A126C
:100EE000031D742F1030880006303D028A110A124B
:100EF000031D7C2F2030880007303D028A110A1222
:100F0000031D842F4030880008303D028A110A12E8
:100F1000031D8C2F8030880009303D028A110A128F
:100F2000031C932F880109303D028A110A12031D08
:100F30009B2F013085000A303D028A110A12031DE1
:100F4000A32F023085000B303D028A110A12031DC7
:100F5000AB2F043085000C303D028A110A12031DAC
:100F6000B32F0830850009303D028A110A12031898
:100F7000BA2F85010800B001BF01BE01A101A00187
:100F80003208870005308A0104204030870033088A
:100F9000870005308A01042040308700340887002C
:100FA00005308A010420403087003508870005306D
:100FB0008A010420403087003608870005308A0106
:100FC0000420403087003708870005308A0104205C
:100FD000403087003808870005308A0104204030FF
:100FE00087003908870005308A01042040308700D7
:100FF0003A08870005308A010420403087003B080A
:10100000870005308A0104208030870087018A1517
:101010000A125A218A150A12861A11288A150A12EA
:1010200033288A150A12061A18288A150A124A291C
:101030008A150A1286191F288A150A12B4238A15DE
:101040000A12061D242887018A150A12061D2A285D
:101050008A013D288A150A12061C31288A150A12AF
:10106000D1298A01BB2F0130A500F4308A01052067
:101070008A150A12861A3F288A150A123328031085
:10108000B20D403032028A150A12031D4A288A1511
:101090000A12B2280310B30D403033028A150A1227
:1010A000031D55288A150A12B2280310B40D4030CA
:1010B00034028A150A12031D60288A150A12B22802
:1010C0000310B50D403035028A150A12031D6B2836
:1010D0008A150A12B2280310B60D403036028A155E
:1010E0000A12031D76288A150A12B2280310B70DBA
:1010F000403037028A150A12031D81288A150A1208
:10110000B2280310B80D403038028A150A12031DA8
:101110008C288A150A12B2280310B90D4030390202
:101120008A150A12031D97288A150A12B22803107D
:10113000BA0D40303A028A150A12031DA2288A15F8
:101140000A12B2280310BB0D40303B028A150A1266
:10115000031DAD288A150A12B2288A150A125A21CF
:101160008A01BB2F403032028A150A12031DBA28A9
:101170000130B300403032028A150A12031DC12823
:10118000B201403033028A150A12031DC92801300A
:10119000B400403033028A150A12031DD028B3016F
:1011A000403034028A150A12031DD8280130B500D8
:1011B000403034028A150A12031DDF28B401403082
:1011C00035028A150A12031DE7280130B6004030A7
:1011D00035028A150A12031DEE28B5014030360289
:1011E0008A150A12031DF6280130B7004030360276
:1011F0008A150A12031DFD28B601403037028A15F0
:101200000A12031D05290130B800403037028A1543
:101210000A12031D0C29B701403038028A150A1240
:10122000031D14290130B900403038028A150A1212
:10123000031D1B29B801403039028A150A12031D0B
:1012400023290130BA00403039028A150A12031DE1
:101250002A29B90140303A028A150A12031D32299F
:101260000130BB0040303A028A150A12031D3929A9
:10127000BA0140303B028A150A12031D4129013090
:10128000B20040303B028A150A12031D4829BB01F7
:101290008A01BB2FBF010130A500F4308A0105206F
:1012A0008A150A12061A57298A150A124A29BD0AEE
:1012B0008A01BB2F0D303D028A150A12031D6229D7
:1012C0000130BD0001303D028A150A12031D6A2952
:1012D0000130880002303D028A150A12031D72296E
:1012E0000230880003303D028A150A12031D7A2954
:1012F0000430880004303D028A150A12031D822939
:101300000830880005303D028A150A12031D8A291B
:101310001030880006303D028A150A12031D9229FA
:101320002030880007303D028A150A12031D9A29D1
:101330004030880008303D028A150A12031DA22998
:101340008030880009303D028A150A12031CA92941
:10135000880109303D028A150A12031DB1290130A6
:1013600085000A303D028A150A12031DB929023090
:1013700085000B303D028A150A12031DC129043075
:1013800085000C303D028A150A12031DC929083058
:10139000850009303D028A150A120318D0298501FB
:1013A000080087010A308A01042040308700870145
:1013B0000A308A01042040308700870109308A0101
:1013C00004204030870087010A308A010420403021
:1013D000870087010A308A01042040308700870196
:1013E0000A308A0104204030870087010A308A01D0
:1013F00004204030870087010A308A0104204030F1
:10140000870087010A308A01042040308700870165
:101410002230A300FE308A0112208030870087012D
:101420008A150A1249233D3030028A150A12031D1B
:101430001C2A8A150A12342ABF0A32303F028A1542
:101440000A12031D242AB00A32303F028A150A12FA
:10145000031D2B2ABF018A150A120618312A8A0198
:101460003D288A150A12D129B001BF01BE01A10190
:10147000A0010310B20D403032028A150A12031D7A
:10148000442A8A150A12A92A0310B30D40303302E8
:101490008A150A12031D4F2A8A150A12A92A031057
:1014A000B40D403034028A150A12031D5A2A8A15D7
:1014B0000A12A92A0310B50D403035028A150A1206
:1014C000031D652A8A150A12A92A0310B60D403099
:1014D00036028A150A12031D702A8A150A12A92AD1
:1014E0000310B70D403037028A150A12031D7B2AFC
:1014F0008A150A12A92A0310B80D403038028A153D
:101500000A12031D862A8A150A12A92A0310B90D88
:10151000403039028A150A12031D912A8A150A12CF
:10152000A92A0310BA0D40303A028A150A12031D87
:101530009C2A8A150A12A92A0310BB0D40303B02CF
:101540008A150A12031DA72A8A150A12A92A8A01D6
:10155000222D403032028A150A12031DB12A0130B1
:10156000B300403032028A150A12031DB82AB201B4
:10157000403033028A150A12031DC02A0130B4001C
:10158000403033028A150A12031DC72AB3014030C6
:1015900034028A150A12031DCF2A0130B5004030EB
:1015A00034028A150A12031DD62AB40140303502CE
:1015B0008A150A12031DDE2A0130B60040303502BA
:1015C0008A150A12031DE52AB501403036028A1534
:1015D0000A12031DED2A0130B700403036028A1589
:1015E0000A12031DF42AB601403037028A150A1286
:1015F000031DFC2A0130B800403037028A150A1258
:10160000031D032BB701403038028A150A12031D4F
:101610000B2B0130B900403038028A150A12031D25
:10162000122BB801403039028A150A12031D1A2BF9
:101630000130BA00403039028A150A12031D212BED
:10164000B90140303A028A150A12031D292B0130D4
:10165000BB0040303A028A150A12031D302BBA0132
:1016600040303B028A150A12031D382B0130B200AC
:10167000013005028A150A12031D3F2BBD0A4030B6
:101680003B028A150A12031D462BBB018A150A125A
:10169000D1290D303D028A150A12031D512B01304C
:1016A000BD0001303D028A150A12031D582B880126
:1016B00002303D028A150A12031D5F2B8801033098
:1016C0003D028A150A12031D662B880104303D0273
:1016D0008A150A12031D6D2B880105303D028A15FB
:1016E0000A12031D742B880106303D028A150A1266
:1016F000031D7B2B880107303D028A150A12031D4A
:10170000822B880108303D028A150A12031D892B9D
:10171000880109303D028A150A12031C902B8801AA
:1017200009303D028A150A12031D972B85010A30E4
:101730003D028A150A12031D9E2B85010B303D02C6
:101740008A150A12031DA52B85010C303D028A154E
:101750000A12031DAC2B850109303D028A150A12BD
:101760000318B32B850108000130B200B301B401A6
:10177000B501B601B701B801B901BA01BB01B001A9
:10178000BF01BE010130BD008701880180308700A4
:0417900087010800C5
:02400E00723FFF
:00000001FF
